:100000000C9436040C946E040C946E040C946E04E0
:100010000C946E040C946E040C946E040C946E0498
:100020000C946E040C946E040C94BD150C94FF1487
:100030000C94711D0C946E040C946E040C946E045C
:100040000C946E040C946E040C946E040C946E0468
:100050000C94FB1F0C94241D0C946E040C946E04E1
:100060000C946E040C946E040C946E040C946E0448
:100070000C946E040C946E040C946E040C946E0438
:100080000C946E040C946E040C946E040C946E0428
:100090000C946E040C946E040C946E040C946E0418
:1000A0000C946E040C946E040C946E0407090A09F7
:1000B00045096E0975098009830983098309D80AEE
:1000C000D80A3E0A410A450A6B0A8D0A900A930A29
:1000D000B70A6D0C6F0CC80C770CAF0C870CD50CE5
:1000E000390DAD0D410D0B0D0F0D450D120D480DC8
:1000F000530D1D0DA30D210D570D250D5B0D850D08
:10010000290D5F0D8F0D2F0D650D6F0D160D4C0D0B
:10011000190D4F0D340D6A0D7B0D9B0D9D0D070DB7
:100120003D0DB60DDF0DE50DD00DD60DEB0DF10D2E
:10013000F70D2E0E540E590E5E0E630E680E6D0EE8
:10014000720E770E7C0E810E410F410F740F740FEB
:10015000F30F11101211121116108A109B109B1020
:100160000F133613E7143613E7148213A513E7149D
:100170009B14AB141E0F0500047F3F1F64321464F0
:100180003214783C1E1E140A050000000000000016
:10019000000000000000000000000000000000005F
:1001A000000000000000000000000000007E0F00C2
:1001B000D4FFFFFFC700000078000000000000002F
:1001C000002A2B28000000000000000000000000B2
:1001D0000000000029000000002C1E3420212224F1
:1001E000342627252E362D3738271E1F202122237F
:1001F0002425263333362E37381F04050607080911
:100200000A0B0C0D0E0F10111213141516171819D6
:100210001A1B1C1D2F3130232D3504050607080934
:100220000A0B0C0D0E0F10111213141516171819B6
:100230001A1B1C1D2F3130354C05010902A1018507
:10024000020901A1000509190129081500250195D8
:1002500008750181020501093009311581257F9555
:10026000027508810609381581257F950175088179
:1002700006050C0A38021581257F9501750881064F
:10028000C0C005010980A101850319012AB7001525
:100290000126B700950175108100C0050C0901A168
:1002A00001850419012AA002150126A002950175F5
:1002B000108100C00660FF0961A1010962150026D6
:1002C000FF009520750881020963150026FF00953F
:1002D0002075089102C005010906A101050719E072
:1002E00029E715002501950875018102950175081A
:1002F00081010507190029FF150026FF00950675E5
:1003000008810005081901290515002501950575C5
:10031000019102950175039101C009025B0003017F
:1003200000A0FA09040000010301010009211101E4
:1003300000012244000705810308000109040100AF
:10034000020300000009211101000122220007051B
:1003500082032000010705030320000109040200B5
:100360000103000000092111010001227B000705A3
:1003700084032000011201000200000008E1AC49E2
:10038000540100010200011003540069007400616F
:10039000006E003600300000001803410063006565
:1003A000006B006500790062006F006100720064FC
:1003B0000000000403090400000000000000000029
:1003C000000001010203040506080A0C0F111418AD
:1003D0001C2024292E33393F464C535B626A7179C5
:1003E000818A929AA2AAB2B9C1C8CFD5DCE1E7EB63
:1003F000F0F4F7FAFCFDFEFFFEFDFCFAF7F4F0EB7B
:10040000E7E1DCD5CFC8C1B9B2AAA29A928A8179B4
:10041000716A625B534C463F39332E2924201C18E5
:1004200014110F0C0A080605040302010100000064
:100430000000000000000029001E001F0020002115
:10044000002200230024002500260027002D002E76
:10045000002A002B0014001A000800150017001CC9
:100460000018000C00120013002F0030003100397A
:100470000004001600070009000A000B000D000E22
:10048000000F003300340000002800E10000001DD0
:10049000001B00060019000500110010003600378F
:1004A000003800E5000000E000E300E2000000008A
:1004B0000000002C00000000000000E600E7002122
:1004C00052E40001000100010001000100010001EF
:1004D0000001000100010001000100010001000114
:1004E0000001000100010001000100010001000104
:1004F00000010001000100010001000100010001F4
:1005000000010001000100010001000100010001E3
:1005100000010000000100010000000100010001D5
:1005200000010001000100010001000100010001C3
:1005300000000001000100010000000000000001B7
:1005400000000000000000010001000100010001A6
:100550000001000100010001000100010001000193
:100560000001000100010001000100010001000183
:100570000001000100010001000100010001000173
:100580000001000100010001000100010001000163
:100590000001000100010001000100010001000054
:1005A0000001000100000001000100010001000144
:1005B0000001000100010001000100010000000134
:1005C0000001000100000000000000010000000028
:1005D0000000000100010001000100010001000114
:1005E0000001000100010001000100010001000103
:1005F00000010001000100010001000100010001F3
:1006000000010001000100010001000100010001E2
:1006100000010001000100010001000100010001D2
:1006200000010001000100010001000000010001C3
:1006300000000001000100010001000100010001B3
:1006400000010001000100010000000100010001A3
:100650000000000000000001000000000000000198
:10066000000100010001002223252628292A2C2D23
:100670002F3032333536383A3B3D3E4042434547D2
:10068000494A4C4E5051535557595A5C5E6062640A
:100690006668696B6D6F71737577797B7D7F818318
:1006A0008587898A8C8E90929496989A9C9E9FA119
:1006B000A3A5A7A8AAACAEAFB1B3B4B6B8B9BBBC3A
:1006C000BEBFC1C2C3C5C6C7C9CACBCCCDCED0D1AF
:1006D000D2D2D3D4D5D6D7D7D8D9D9DADADBDBDBA7
:1006E000DCDCDCDCDCDDDDDDDDDCDCDCDCDCDBDB48
:1006F000DBDADAD9D9D8D7D7D6D5D4D3D2D2D1D09C
:10070000CECDCCCBCAC9C7C6C5C3C2C1BFBEBCBB98
:10071000B9B8B6B4B3B1AFAEACAAA8A7A5A3A19F10
:100720009E9C9A98969492908E8C8A8987858381D4
:100730007F7D7B79777573716F6D6B6968666462B5
:10074000605E5C5A5957555351504E4C4A49474583
:100750004342403E3D3B3A3836353332302F2D2C24
:100760002A29282625232200010101010101010176
:100770000102020202020202020203030303030354
:100780000303040404040404040505050505060622
:1007900006060607070707070808080809090909E0
:1007A0000A0A0A0B0B0B0C0C0C0D0D0D0E0E0E0F86
:1007B0000F0F101011111112121313141415151616
:1007C000161717181819191A1A1B1B1C1D1D1E1E87
:1007D0001F202021222223242425262627282929D8
:1007E0002A2B2C2D2D2E2F30313232333435363703
:1007F00038393A3B3C3D3E3F404142434445464701
:1008000048494A4C4D4E4F50515354555658595AD9
:100810005B5D5E5F616264656668696B6C6D6F707D
:1008200072737577787A7B7D7E8082838587888AEC
:100830008C8E8F91939596989A9C9EA0A2A3A5A723
:10084000A9ABADAFB1B3B5B7BABCBEC0C2C4C6C91F
:10085000CBCDCFD1D4D6D8DBDDDFE2E4E7E9EBEED8
:10086000F0F3F5F8FAFDFFFFAA7F554011241FBEF3
:10087000CFEFDAE0DEBFCDBF04B603FE18C0809133
:10088000BE029091BF02A091C002B091C102873018
:10089000904BA740B04B59F41092BE021092BF0289
:1008A0001092C0021092C102E0E0F8E3099511E055
:1008B000A0E0B1E0E0EEF8E502C005900D92A83AA4
:1008C000B107D9F722E0A8EAB1E001C01D92AE3B22
:1008D000B207E1F70E9470040C946E2C0C94000097
:1008E000A6E2B0E0E6E7F4E00C94E62B85B780687A
:1008F00085BF85B7806885BF84B7877F84BF0FB603
:10090000F894A895809160008861809360001092AF
:1009100060000FBE90E080E80FB6F894809361000D
:10092000909361000FBE81E08093110186ED96E106
:100930009093A9018093A8010E9443150E9462151B
:100940008091E20084608093E20078948091DE01DF
:100950008823A1F01091E9001F709091EC00892F7D
:10096000817090FD80E8182B1092E9008091E800DA
:1009700083FD0E9427121F701093E90082E084BD5E
:1009800093E095BD9AEF97BD80936E000E943A1E4A
:10099000811102C00E94BD1F01E211E0D8018D91BA
:1009A0008D018F3F11F00E94E317B1E006321B0763
:1009B000A9F706E211E0B4E3EB2EB1E0FB2EF8015B
:1009C00081918F018F3F11F00E94E317E016F1062D
:1009D000B1F78AE0E7ECF1E0DF01282F1D922A95BC
:1009E000E9F7EAEAF1E0DF011D928A95E9F780E094
:1009F00090E00E94CB2A853E9E4F21F40E943A1E31
:100A0000811163C065EE7EEF80E090E00E94FF2AD6
:100A100060E082E090E00E94E12A81E08093B401EE
:100A200061E083E090E00E94E12A60E074E184E00C
:100A300090E00E94FF2A60E086E090E00E94E12AB8
:100A400060E087E090E00E94E12A40E050E0BA01D7
:100A500088E090E00E94F32A60E083E290E00E9448
:100A6000E12A60E08CE090E00E94E12A60E08DE005
:100A700090E00E94E12A19821A821B821C821D8248
:100A80001E821F82188648E050E067E170E0CE01C8
:100A900001960E94D12A40E050E0BA018FE190E037
:100AA0000E94F32A80E00E941B1E0E94BD1F40E0AE
:100AB00050E0BA018FE090E00E94F32A40E050E05D
:100AC000BA0183E190E00E94F32A82E090E00E9464
:100AD000BD2A8093BB0184E090E00E94CB2A9093D2
:100AE000B7018093B6010E94FA17EFEFF6E721E015
:100AF000E150F0402040E1F700C000000E94FA17EA
:100B00008091C70180FF08C06FEF7FEF80E090E029
:100B10000E94FF2A0E94001D83E090E00E94BD2AEF
:100B20000E946021279A2F988AE08093800089E1B3
:100B3000809381008FEF9FEF9093870080938600D2
:100B40000E94D1248091420281FF0BC01092450285
:100B5000109244021092430280916F008160809352
:100B60006F000E94D1248091B80181117FC088E07C
:100B700090E00E94C52A4B015C0183E290E00E9454
:100B8000BD2A282F30E040E050E060E070E080E0D7
:100B900090E000E20E941D2C282939294A295B296E
:100BA0002093B6023093B7024093B8025093B90233
:100BB0006093BA027093BB028093BC029093BD0213
:100BC0002C7F09F041C025E02093B6021092B702B5
:100BD0003FEF3093B8023093B9021092BA0230E07E
:100BE0004FEF5FEF60E00E94012888E090E00E94F4
:100BF000C52A6B017C0183E290E00E94BD2A282F68
:100C000030E040E050E060E070E080E090E00E9482
:100C10001D2CB22FA32FF42FE52F5B019701860126
:100C2000BC29A12BF22BE32BB093B602A093B70201
:100C3000F093B802E093B9026093BA02B092BB029B
:100C40008093BC029093BD020E94ED271092950202
:100C50000E94871C8091B60280FF05C060E08695E7
:100C600086950E942F2981E08093B80184E091E06D
:100C700090936B0280936A02552453942224239408
:100C80008E010F5F1F4F8091DE01853009F061C03A
:100C90008091DE01853009F04DC08091DE01843005
:100CA00009F43AC080E00E9492241092950280914B
:100CB000BA0181110DC05092BA018091B602982FED
:100CC00091709093B9018E7F8093B6020E940F2598
:100CD00010926E0288E190E0A0E40FB6F894A89517
:100CE000809360000FBEA093600083B7817F846013
:100CF00083BF83B7816083BF7894889583B78E7FE5
:100D000083BF0FB6F894A8958091600088618093A6
:100D10006000109260000FBE0E94FA17E7ECF1E04D
:100D200081919191892B09F04CC4B1E0E13DFB0721
:100D3000B9F7AECF0E9486210E94D1240E94091EDD
:100D40001092BA018091B90181110E9474290E9408
:100D5000F8240E94FA17FCEBEF2EF1E0FF2EA7EC2F
:100D60006A2EA1E07A2ED301F701219131918D9164
:100D70009D918227932721E0E63CF20719F0892B09
:100D8000A1F305C0892B19F40E94D8193EC0412C4B
:100D9000D3018D909D903D01F701A080B180A824E2
:100DA000B924A114B10441F1312CCC24C394D12C29
:100DB000C5018C219D21892BB1F039A24AA20E9444
:100DC000651D9CA38BA32DA291E094012C213D21B4
:100DD000232B09F490E09EA349A15AA16BA17CA109
:100DE0008DA10E94BB293394CC0CDD1CFEE03F1288
:100DF000DFCFD7018D929C924394B2E0EB0EF11CB1
:100E0000E5E04E12C5CF0E94591D809195028823BE
:100E100009F4ABC080919402E091B602E695E695A4
:100E2000E81BE0939002823059F4F0E0EB57FE4F5C
:100E3000E491EE2EF12C6FECC62E63E2D62E70C03C
:100E4000863059F4F0E0EE57FE4FE491EE2EF12C8F
:100E50005FEBC52E53E2D52E63C0893061F4E69571
:100E6000F0E0E158FE4FE491EE2EF12C4DE0C42E5F
:100E700047E2D42E55C08F3061F4E695F0E0E45897
:100E8000FE4FE491EE2EF12C3CEAC32E36E2D32E37
:100E900047C0853159F4F0E0E758FE4FE491EE2E5B
:100EA000F12C20E6C22E26E2D22E3AC08831F9F08B
:100EB000833249F4E7E7F1E0E590F49092EAC92E35
:100EC00093E2D92E2DC08432D1F0853209F58E2FD0
:100ED00063E00E94882BE92FF0E0EC58FE4FE4918C
:100EE000EE2EF12C87E2C82E85E2D82E19C0A8E29A
:100EF000EA2EF12CB8EECB2EB5E2DB2E11C0E4EFDA
:100F0000EE2EFF24F394F9EBCF2EF5E2DF2E08C08E
:100F100060EDE62E67E0F62E71EAC72E73E2D72E5B
:100F200080919102882361F0109291020E94651DC8
:100F300090938F0280938E021092930210929202ED
:100F40000E94651DE0918E02F0918F028E1B9F0B17
:100F50008F3F9F4750F4EE0EFF1EF0928F02E092FB
:100F60008E028EE892E0F601099586E0EFE5F2E068
:100F7000D80101900D928A95E1F7B0906002F0904F
:100F80006102C0906202D0906302E090640210920D
:100F90006102109262021092630210926402F110D8
:100FA00003C0CC2009F44BC080915D0290915E0299
:100FB0000E944A1D9C0190915802992309F427C36D
:100FC00025313105E0F19F3F19F09F5F9093580262
:100FD000FF2061F00E94231F1F1414F491E001C050
:100FE0009FEF899F802D112480936102CC2061F0B6
:100FF0000E94231F1C1414F09FEF01C091E0899FF1
:10100000802D112480936202809161028823B9F0BF
:10101000A0906202AA2099F00E94431F882319F031
:101020008093610202C0509261028A2D0E94431F88
:10103000882319F08093620202C050926202D1109C
:1010400003C0EE2009F44BC080915B0290915C02DA
:101050000E944A1D9C0190915902992309F4DCC217
:1010600021353105E0F19F3F19F09F5F90935902C0
:10107000DD2061F00E94011F1D1414F491E001C0F5
:101080009FEF899F802D112480936302EE2061F0F1
:101090000E94011F1E1414F09FEF01C091E0899F70
:1010A000802D112480936402809163028823B9F01B
:1010B000A0906402AA2099F00E94431F882319F08F
:1010C0008093630202C0509263028A2D0E94431FE4
:1010D000882319F08093640202C0509264028091C8
:1010E00060028B111AC080916102882311F08F1168
:1010F00014C080916202882311F08C110EC080917F
:101100006402882311F08E1108C090916302992324
:1011100031F081E09D1104C002C081E001C080E097
:1011200080FD15C08091610281110FC08091620223
:1011300081110BC080916302811107C081E0909101
:101140006402911103C080E001C081E080FD0E9433
:10115000D71EBA82FB82CC82DD82EE8286E0F80165
:10116000AFE5B2E001900D928A95E1F70E94091E69
:101170009091C601891721F08093C6010E94591DE4
:101180008091DE01843009F07ECD83E08093E90018
:101190008091E80082FF77CD8091E80085FF21C033
:1011A0000E94A31681111BC050E2E52EF12C6801AC
:1011B00009C08091F100D6018D936D01B1E0EB1A69
:1011C000F10869F08091E80085FDF3CF8091E80097
:1011D0008B778093E8000E94A316882399F391E00F
:1011E00001C090E08091E8008B778093E80099231C
:1011F00009F449CD2981822F90E0FC013197E33138
:10120000F10508F0D5C1EA5AFF4F0C94CA2B1A8297
:101210008CE039C18A81823009F4F0C150F4813008
:1012200009F0C6C10E94591D9B838C837D836E8308
:10123000C1C1833041F0843009F0BAC11B821C82E5
:101240001D821E82B7C16B81D80180E090E0262FFD
:1012500030E0A901480F591F4530510508F0AAC1D7
:10126000E62FE80FF0E0EE0FFF1FE953FE4F40813D
:10127000518113965C93139714964C93149701968F
:1012800012968E30910529F795C18A81823019F026
:10129000853051F08DC16B817C818D819E810E9452
:1012A000D02B0E94161E86C18091420280FF03C08F
:1012B0000E94AC2402C00E94B9248091B60280FF33
:1012C0000AC08091B6028E7F8093B602109295027A
:1012D0000E940F256FC10E9474296CC14C816B81E3
:1012E0008A810E94CD1F9D8390C12D813E8132272E
:1012F000232732274C816B818A810E94611F5AC14A
:101300000E94881F57C18A818130E1F52830F1F0B1
:10131000293099F18B81813019F0823071F04AC106
:101320008C81E3E08E9FC00111246FEF70E00E947A
:10133000A22B862F0E9492243DC18C81811103C073
:101340000E94672437C10E947D2434C18B81813083
:1013500041F0823009F02EC1809142028695817061
:1013600078C080914202869586958695FFEF8F9F83
:10137000C001112463E070E05DC0809142020E94D0
:10138000612418C1823009F013C12830B9F1293025
:1013900009F461C08B818230F9F098F4813009F052
:1013A00009C18C812FEF829FC00111246FEF70E083
:1013B0000E94A22B462F20E06091B8028091B702D4
:1013C0001AC08330A1F0843009F0F4C020E04091CD
:1013D000B9026D818C810FC08C81882309F471CF93
:1013E0000E94742960E08C810E942F29E3C08C81C7
:1013F0008093BA02DFC00E946A28DCC08B818230F1
:10140000E9F060F4813009F0D5C08091B902AFEF06
:101410008A9FC00111246FEF70E00CC08330B9F0D7
:10142000843009F0C7C08091B7028C838091B802E4
:101430008D83C0C00E94A22B6C83BCC08091B60279
:1014400080FF03C08695869504C080E002C080912D
:10145000BA028C83AFC02091B6023091B70240919E
:10146000B8025091B9026091BA027091BB028091AA
:10147000BC029091BD020E9401289CC0B0E1BA83D9
:1014800099C05A8288EA8B8395C0EA80FB80FE244B
:10149000EF24FE24CC80D12C5801C701885A9D4FDF
:1014A0009501201B310B2C153D0508F083C0E8EA9F
:1014B000EE16E1E0FE0630F40E94BD2AD501149636
:1014C0008C9302C0F5011482FFEFEF1AFF0A2FEF91
:1014D000A21AB20AE2CFEA80FB80FE24EF24FE24A7
:1014E000CC80D12C5801C701885A9D4F9501201BF3
:1014F000310B2C153D0508F05DC0A8EAEA16A1E005
:10150000FA0620F4F50164810E94E12AFFEFEF1A48
:10151000FF0A2FEFA21AB20AE6CF0E94511F4AC05B
:1015200084E08A8347C0EA80FB80FE24EF24FE2407
:10153000CC80D12C5801C70188969501201B310B16
:101540002C153D05B8F5A0E3EA16A2E0FA0628F44A
:101550000E94BD2AF501848303C0D50114961C9214
:10156000BFEFEB1AFB0AEFEFAE1ABE0AE4CFEA8038
:10157000FB80FE24EF24FE24CC80D12C5801C7012F
:1015800088969501201B310B2C153D0598F4F0E34E
:10159000EF16F2E0FF0628F4D50114966C910E9434
:1015A000E12ABFEFEB1AFB0AEFEFAE1ABE0AE7CF54
:1015B0008FEF898340E250E0B80182E00E94AE1CC8
:1015C00062CB8091DD01882309F462CBE0E1E9BDC3
:1015D000F2E1F9BD09B400FEFDCF8091D8008F7D06
:1015E0008093D8008091E00082608093E000809139
:1015F000E00081FDFCCF0E9486214ACB87E290E08B
:101600000E94BD2A1B821C821D828E83D3CF2B3069
:10161000310508F0DACC13CD2B30310508F025CD9B
:101620005ECDA8E0B0E0E7E1FBE00C94E62BFC0126
:101630008481882309F447C67F0121E040815181DC
:101640006281738195810E9496298C01F7019581B1
:10165000992309F4B4C1980137572038310508F0AF
:1016600032C1003108F0DCC28FEF93E00E94BD2A46
:101670008111D6C238E5A32E32E0B32E002379F0D3
:10168000A114F4E0BF0609F4CBC2C5010E94BD2A33
:10169000811101C001502FEFA21AB20AEFCFCE0183
:1016A00001962C0188E0F20111928A95E9F72AE06F
:1016B000322E85010F5F1F4FC5010E94BD2A89830D
:1016C0001A82882309F4ACC2813009F041C0650157
:1016D000F2E0CF0ED11CC8010E94BD2A8A83882364
:1016E00009F49EC29FEF980F933060F423E0A20E9E
:1016F000B11CC6010E94BD2A8B83882309F490C2C5
:101700001C8229C0843031F54E0133E0830E911CD8
:1017100002E010E056018FEFA81AB80AC6010E9435
:10172000BD2AF40181934F01882309F479C28C37D3
:1017300041F4E2E0F0E0EC0FFD1FE00FF11F10823A
:101740000AC00F5F1F4F65010730110519F768C206
:10175000580101C056018201F8012081222309F4B9
:10176000A8CF213009F053C08181813081F4680114
:10177000F2E0CF0ED11CF8018281893319F460E5C3
:1017800070E002C060E070E00E94892315C08230E2
:1017900049F46801F2E0CF0ED11CF80182810E9469
:1017A000F0220AC0833051F46801F2E0CF0ED11C60
:1017B000F80182810E949622860182C0843019F04D
:1017C0000F5F1F4F7DC0F80122810E5F1F4F80E029
:1017D00090E030E0205331092A30310568F4389E1A
:1017E000A001399E500D1124C901840F951F0F5F70
:1017F0001F4FF8012081EDCF009709F461C0EFE998
:10180000FFE03197F1F700C000000197F5CFE22F1C
:10181000F0E0E754FE4F2490822F869586958695BA
:1018200090E0FC01E755FE4F64902770712C022E6A
:1018300002C0759467940A94E2F7F1E06F2277246E
:10184000FC01E756FE4F8490912C022E02C0959425
:1018500087940A94E2F731E083229924FC01E75748
:10186000FE4FC490D12C02C0D594C7942A95E2F7BC
:1018700081E0C822DD246114710419F081EE0E9418
:10188000F0228114910419F086EE0E94F02260E0AB
:1018900070E0822D0E9489238114910419F086EE54
:1018A0000E9496226114710419F081EE0E94962222
:1018B000C114D10429F060E070E08CE20E94892319
:1018C0000F5F1F4F49CFF801F857E730F10508F0D7
:1018D00076C0E759FF4F0C94CA2B83E001C080E02B
:1018E0000E949224809142020E94612499C18091B9
:1018F0004202982F96959695969549F1915E990F8B
:10190000990F990F8770892B8093420214C0909190
:101910004202892F8695869586958F5F8F71977085
:10192000843008F03FC0880F880F880F892B809380
:10193000420280914202887F91E009F490E0809118
:10194000420290FB80F9809342020E9461248091C0
:1019500042028695869586950E94742061C12091E9
:101960004202822F869586958695482F50E0433017
:10197000510554F48F5F982F990F990F990F822F6B
:101980008770892B80934202809142028160DBCF75
:101990008091420280FF03C00E94AC2441C10E949A
:1019A000B9243EC190934202C4CF8091420281FF8C
:1019B00003C00E94672434C10E947D2431C1F80114
:1019C000E851FC47E730F10508F4E6C0992309F433
:1019D00053C410926702980130572332310508F042
:1019E0000CC184E090E00E94CB2A9093B7018093D1
:1019F000B601F801E150F047E232F10520F4E05978
:101A0000FF4F0C94CA2B8091B6018160ACC08091CD
:101A1000B7018860B4C08091B6018260A4C0809193
:101A2000B60120C08091B60188609DC08091B70149
:101A30001EC08091B7018260A2C08091B601806112
:101A400092C08091B60180628EC08091B6018064A0
:101A50008AC00E9486218091B601806884C08091EE
:101A6000B601886084607FC08091B7018260816028
:101A700086C08091B6018E7F76C08091B701877F46
:101A80007EC08091B6018D7F6EC08091B60120C06E
:101A90008091B601877F67C08091B7011EC0809199
:101AA000B7018D7F6CC08091B6018F7E5CC0809144
:101AB000B6018F7D58C08091B6018F7B54C00E94C3
:101AC00086218091B6018F774EC08091B601877FC5
:101AD0008B7F49C08091B7018D7F8E7F50C08091F0
:101AE000B60182FB222720F991E0922790FB82F930
:101AF00090FB83F938C08091B701982F9095917031
:101B00008E7F892B90FB81F93AC08091B60186FBCC
:101B1000222720F991E0922790FB86F924C00E94A9
:101B200086218091B60187FB222720F991E0922738
:101B300090FB87F918C061E001C060E08EE090E0A2
:101B40000E94E12A1EC08091B60184FB222720F961
:101B500091E0922790FB84F906C08091B601982FFE
:101B6000909590FB80F98093B6010BC08091B701EE
:101B700083FB222720F991E0922790FB83F9809341
:101B8000B7016091B6017091B70184E090E00E94C6
:101B9000FF2A0E94862144C0EE56FF4F0C94CA2BA8
:101BA00006E221EE41EE6AE17CE705C007E225EEA0
:101BB00045EE6BE17CE7C7010E94531E31C006E28F
:101BC00021EE40EE68E17CE7F6CF07E225EE44EE39
:101BD00069E17CE7F0CF06E221EE42EE6CE17CE7C2
:101BE000EACF07E225EE46EE6DE17CE7E4CF08E2BE
:101BF00021E045EE6EE17CE7DECF809134020631D4
:101C0000FCE71F07F9F48A7A91E009F490E09093D9
:101C1000D10181112FC389E20E94A61D0E94031ADF
:101C200080912902877009F44EC3F70185818823CA
:101C300009F449C38091B70182FF45C382E00E9445
:101C40003D1A41C38272F801E052F847EB30F105CA
:101C500008F05CC0E756FF4F0C94CA2B8091B60287
:101C600080FF19C0282F2E7F2093B6023091B70233
:101C70004091B8025091B9026091BA027091BB02D2
:101C80008091BC029091BD020E94012810929502A1
:101C90000E940F25C5CF81608093B60261E08695D2
:101CA00086950E942F29BCCF882329F00E947F2986
:101CB000B7CF8823D9F30E948A29B2CF882329F08D
:101CC0000E941B29ADCF8823D9F30E942529A8CFD4
:101CD000882329F00E940129A3CF8823D9F30E94E9
:101CE0000E299ECF882329F00E94E72899CF8823C8
:101CF000D9F30E94F42894CF882329F00E94272842
:101D00008FCF8823D9F30E9441288ACF0737FCE779
:101D10001F0711F481E0CCC208372CE7120709F441
:101D2000C6C29801205E324520323105A8F49111D7
:101D300015C00F7181E090E0FC0102C0EE0FFF1FA3
:101D40000A95E2F78F016E2F83E090E00E94E12A6E
:101D5000802F0E94602164CF9923E9F10330FCE7D2
:101D60001F0729F148F401153CE7130791F00130F2
:101D70008CE7180711F12FC00B359CE7190741F1CB
:101D80000C35ECE71E07E1F00A351C4721F581E030
:101D900020C00E9486212FEF34E38CE02150304098
:101DA0008040E1F700C000000E94001D39CF6FEFB6
:101DB0007FEF80E090E00E94FF2A0E944B2A30CF04
:101DC0008091B70182FB882780F991E0892701C0C3
:101DD00080E00E94541AF7018581008111818823D7
:101DE00049F0C8010E949F20D82E682FC8010E9488
:101DF0000F2104C0C8010E94DB20D82EB8018D2D10
:101E00000E94AD180E94BB18D82E192FA82EF701DA
:101E10000581C680C2949FE0C92280912902877003
:101E200001F10023F1F0812F807F803469F080E29E
:101E30008D0D8830B0F0812F807E803229F4F1E062
:101E4000FD1578F4CC2069F08091B70182FF09C0BC
:101E500082E00E943D1A809129028770BB24B394CE
:101E60008111B12C912E92948FE09822892D90E0CF
:101E70008C30910508F0D6C1FC01EC55FF4F0C9455
:101E8000CA2B812F807F1F70882311F01295107F3D
:101E90000023B9F0112309F4B3C180E28D0D88301D
:101EA00010F0A11006C090913402192B1093340247
:101EB00005C090912B02192B10932B020E94031A3C
:101EC0009FC18D2D0E949622112309F4ABC180E29F
:101ED0008D0D883088F1AA2079F1109590912B0210
:101EE000192310932B022BC0812F807F1F7080320B
:101EF00011F01295107F8D2DAA2029F021E0A21655
:101F000009F44CC057C08091B70182FD1BC000236B
:101F100069F0112339F090913402192B1093340297
:101F20000E94031A80E00E94F0227CC180E00E949F
:101F30009622112309F476C1812F0E94FC190E9478
:101F4000031A70C1002381F0CC20C1F131E0C3122B
:101F500069C190912A02812F8923181709F462C15F
:101F6000192B10932A025EC1C1105CC1812F0E94FF
:101F7000AD2180912A02912F982329F0912F9095DD
:101F8000892380932A022091D201812F822309F490
:101F900049C1109521232093D20144C1002329F087
:101FA00085E08C1508F43EC109C094E09C1508F446
:101FB00039C115C0002331F0C11022C1812F0E9408
:101FC000B42130C1CC2059F0893309F028C1EFEF9A
:101FD000F7EE23E0E150F0402040E1F71EC1812FF1
:101FE0000E94AD211FC1812F86958695837019F0BF
:101FF000813061F017C1002321F08D2D912F937056
:1020000002C080E090E00E94E41D12C1002321F094
:102010008D2D912F937002C080E090E00E94BF1D33
:1020200007C1602F8D2D0E94BE2102C1812F8370B8
:10203000A9F50111FBC04D2D429546954770440FFF
:10204000440F8D2D8F7090E09C01042E01C0220F53
:102050000A94EAF7D4FE08C08FE090E001C0880F30
:102060004A95EAF7809501C080E0169516951370A1
:10207000123069F088F49091B401113019F0822B7C
:10208000892302C0922B892B0E946021CFC0822B12
:102090009091B4018927F8CF822BF6CF002319F055
:1020A000812F817001C08695882309F4BFC04D2D12
:1020B000429546954770440F440F8D2D8F7090E0E8
:1020C0009C01042E01C0220F0A94EAF7D4FE08C036
:1020D0008FE090E001C0880F4A95EAF7809501C033
:1020E00080E0169516951370123059F078F490919F
:1020F000B501113019F0822B892309C0922B892B4D
:1021000006C0822B9091B501892701C0822B0E94C5
:1021100044218CC01F70002339F0812F0E9454216C
:102120008D2D0E94B42182C08D2D0E94AD21812F62
:102130000E9447217BC08D2D32EFA31681F13A1505
:1021400038F090EFA91659F0E1EFAE1619F154C02E
:10215000F3EFAF1659F124EFA216C1F04DC00023E2
:1021600081F034E03C1508F45DC01F7181E090E01F
:10217000012E01C0880F0A94EAF79091B5018927D2
:1021800020C085E08C1508F44DC0EFCF8091B701D9
:1021900082FD1AC0002329F0812F8F7120C00023F7
:1021A000D9F3812F8F710E9447213CC0002341F059
:1021B0001F7181E0012E01C0880F0A94EAF701C067
:1021C00080E00E9444212EC0002361F0812F8F7196
:1021D00098E0899F900111242360209329020E9496
:1021E000542120C081E00E943D1AE1E0EC15D0F4BA
:1021F00082E00E943D1A16C0002321F0CC2061F23B
:102200008D2D91CECC2069F2893349F4FFEF27EE72
:1022100033E0F15020403040E1F700C000008D2D48
:102220000E94962288EF890D843010F40E94091EC6
:10223000BB20A9F08091290280FD11C0F701158211
:102240008695869586950E945421C7010E94110BA0
:10225000809129028695869586950E94472120E0E7
:10226000F7014081518162817381848195810E944F
:10227000962929C085E3D0CC06318CE7180751F4A4
:102280008091D101811104C089E20E949A1DC6CCBF
:1022900085E3FBCF07372CE7120711F481E00BC071
:1022A00008373CE7130709F03CCD82E004C082E028
:1022B0000E94542102C00E94472143E062E081E075
:1022C0000E94551CADCC2896E2E10C94022C809122
:1022D000E00187FF11C08091E80082FD05C0809178
:1022E000DE018111F8CF11C08091E8008B770BC01F
:1022F0008091DE01882349F08091E80080FFF8CFCB
:102300008091E8008E778093E8000895982F9730A9
:1023100068F59093E900981739F07091EC002091DE
:10232000ED005091F00003C0242F762F50E021FDE6
:1023300002C09F5FECCF3091EB003E7F3093EB000B
:102340003091ED003D7F3093ED003091EB00316036
:102350003093EB007093EC002093ED005093F0006D
:102360002091EE0027FDE5CF80E008958F708093E7
:10237000E90081E008952091E6013091E7012617F8
:10238000370748F06115710539F42091E8002E7780
:102390002093E80001C0B901FC0120E0611571053E
:1023A00079F18091DE018823F1F18530F1F180919E
:1023B000E80083FD3CC08091E80082FD2EC0809142
:1023C000E80080FFEBCF2091F3008091F20090E0D5
:1023D000922B6115710551F08830910538F42191E7
:1023E0002093F100615071090196F3CF21E0089725
:1023F00009F020E08091E8008E778093E800CECF4E
:102400002111CFCF0AC08091DE01882361F0853091
:1024100061F08091E80083FD0AC08091E80082FFAE
:10242000F2CF80E0089582E0089583E0089581E08E
:10243000089543E050E0BC0184E00E94AE1C089582
:1024400046E050E0BC0184E00E94AE1C0895AAE280
:10245000B0E0EDE2F2E10C94F52BE0EEF1E088EE75
:1024600091E02091F10021938E179F07D1F7809181
:10247000E101833009F463C030F4813071F08230BF
:1024800009F4A2C0B9C08A3009F48EC08B3009F4B7
:102490006EC0893009F0B0C020C08091E001813A5F
:1024A00009F0AAC08091E800877F8093E8008091BE
:1024B000E4019091E501892B21F468E084ED91E03D
:1024C00003C060E080E090E070E00E94BB1180916A
:1024D000E8008B778093E8008FC08091E001813223
:1024E00009F08AC08091E4019091E501009719F00C
:1024F000029709F081C08091E800877F8093E8000F
:102500008091E80082FD05C08091DE018111F8CF45
:1025100073C02091F3008091F20090E0922B02971B
:1025200031F48091F100813011F0863021F48091F6
:10253000F10080930F018091E8008B7759C0809162
:10254000E001813A09F058C08091E4019091E501E1
:10255000892B09F051C08091E800877F8093E800C3
:102560008091E80080FFFCCF809110013CC08091F9
:10257000E001813209F040C08091E4019091E501D1
:10258000892BD1F58091E800877F8093E8000E9435
:10259000671181E09091E201911101C080E0809388
:1025A00010010E94862128C08091E001813221F52E
:1025B0008091E800877F8093E8000E9467118091F6
:1025C000E30180930E0118C08091E001813AA1F4EB
:1025D0008091E800877F8093E8008091E80080FF89
:1025E000FCCF80910E018093F1008091E8008E77FE
:1025F0008093E8000E9467118091E80083FFE7C1A3
:102600008091E0019091E101492F50E04A3051055D
:1026100008F0DDC1FA01E055FF4F0C94CA2B803859
:1026200021F0823809F0D3C108C08091DC0190917B
:10263000DD01992389F082600FC08091E4018F70E1
:10264000873008F0C4C18093E9008091EB0085FBDE
:10265000882780F91092E9009091E800977F909385
:10266000E8008093F1001092F10071C1282F2D7FB6
:1026700009F0ADC1882319F0823061F0A8C18091C2
:10268000E201813009F0A3C1933009F080E080932A
:10269000DD012EC08091E20181112AC08091E40108
:1026A0008F702FEF280F263008F091C18093E9003A
:1026B0002091EB0020FF1CC0933021F48091EB00AF
:1026C000806214C09091EB0090619093EB0021E048
:1026D00030E0A90102C0440F551F8A95E2F74093EC
:1026E000EA001092EA008091EB0088608093EB0092
:1026F0001092E9008091E800877F8093E8000E94B3
:10270000671165C1811163C11091E2011F7780914A
:10271000E3008078812B8093E3008091E800877F3D
:102720008093E8000E9467118091E80080FFFCCF51
:102730008091E30080688093E300111102C082E081
:1027400001C083E08093DE0142C18058823008F0EE
:102750003EC12091E2013091E3012C3D53E0350769
:1027600079F583E08A838AE289834FB7F894DE01A2
:10277000139620E03EE051E2E32FF0E05093570043
:10278000E49120FF03C0E295EF703F5FEF708E2F62
:1027900090E0EA3010F0C79601C0C0968D939D93EB
:1027A0002F5F243149F74FBF8091E800877F8093E6
:1027B000E8006AE270E0CE0101960E94BB11B5C04C
:1027C0008091E4019091E501432F55274330510555
:1027D000A9F068F44130510509F408C142305105AF
:1027E00009F0F5C08BE590E0EAE1F3E04BC041323F
:1027F000510529F14232510589F1E9C0C9019927F2
:1028000081309105A1F058F0029709F0E0C0E7E8A7
:10281000F3E0E4918E2F90E0E7E8F3E030C0E3EBE3
:10282000F3E0E4918E2F90E0E3EBF3E028C0E9E9D8
:10283000F3E0E4918E2F90E0E9E9F3E020C08330EB
:10284000910508F0C4C0880F991FFC01E35CFE4F9E
:102850000190F081E02D89E090E014C08330910573
:1028600008F0B5C0FC01EE0FFF1FE95CFE4F0190C0
:10287000F081E02DDC01AC5CBE4F8C9190E00097C4
:1028800009F4A5C02091E800277F2093E80020915B
:10289000E6013091E7018217930708F49C0140E0BC
:1028A0002115310589F18091DE01882309F43DC0AD
:1028B0008530D9F18091E80083FD37C08091E80030
:1028C00082FD2FC08091E80080FFEACF4091F300A5
:1028D0008091F20090E0942B2115310559F0883059
:1028E000910540F444914093F10031962150310913
:1028F0000196F2CF41E0089709F040E08091E800AE
:102900008E778093E800CCCF4111CDCF0AC0809163
:10291000DE01882351F0853041F08091E80083FD8D
:1029200004C08091E80082FFF2CF8091E8008B77AD
:102930008093E8004CC0803809F049C08091E800DD
:10294000877F8093E8008091DF018093F100809180
:10295000E8008E77D2CE81113AC08091E201909149
:10296000E301992702979CF58091E800877F809387
:10297000E8001091E2011093DF010E94671111112C
:1029800006C08091E30087FD02C081E001C084E0C1
:102990008093DE0142E061EC81E00E94861142E218
:1029A00061EC84E00E94861142E261EC82E00E94C8
:1029B000861142E260EC83E00E9486118091DE0184
:1029C000843011F081E001C082E080931101809198
:1029D000E80083FF10C08091E800877F8093E800C3
:1029E0008091EB0080628093EB0005C082E190E073
:1029F000E5E7F3E047CFAA96E3E00C94112C1F9291
:102A00000F920FB60F9211242F933F934F935F9322
:102A10006F937F938F939F93AF93BF93CF93DF93E6
:102A2000EF93FF93C091E900CF708091EC00D82F15
:102A3000D17080FDD0E81092E9008091F000877F8E
:102A40008093F00078940E9427121092E900809100
:102A5000F00088608093F000CD2BCF70C093E90028
:102A6000FF91EF91DF91CF91BF91AF919F918F91A6
:102A70007F916F915F914F913F912F910F900FBE7A
:102A80000F901F901895E8EDF0E080818E7F808395
:102A90001092E2001092DA001092E100A0EEB0E095
:102AA0008C9181608C9380818F77808319BCA7ED96
:102AB000B0E08C918E7F8C9380818F7E808310928A
:102AC000D3010895A0E0B0E0E8E6F5E10C94F02B26
:102AD000C8EDD0E088818F7E8883E7EDF0E08081CB
:102AE0008160808384E082BF81E08093D30188810C
:102AF0008E7F888302EE10E0F80110821092DA00D7
:102B000081EEC82ED12CF601108288818F778883C0
:102B100088818068888388818F7D888319BC109222
:102B2000DE011092DF011092DD011092DC0190EEC7
:102B3000E92EF12CF70180818B7F80838881816071
:102B4000888342E060E080E00E948611F601808187
:102B50008E7F8083F801808181608083808188609E
:102B60008083F70180818E7F808388818061888364
:102B7000CDB7DEB7E8E00C940C2C1F920F920FB685
:102B80000F9211242F933F934F935F936F937F93F3
:102B90008F939F93AF93BF93EF93FF938091E10047
:102BA00082FF09C08091E20082FF05C08091E100B0
:102BB0008B7F8093E1008091DA0080FF2AC08091B2
:102BC000D80080FF26C08091DA008E7F8093DA00E3
:102BD0008091D90080FF18C080E189BD82E189BD64
:102BE00009B400FEFDCF81E08093DE018091D30126
:102BF00081110FC00E9443150E9462158091E2006E
:102C000084608093E20005C019BC1092DE0110922E
:102C1000D3018091E10080FF1AC08091E20080FF23
:102C200016C08091E2008E7F8093E2008091E200E6
:102C300080618093E2008091D80080628093D80008
:102C400019BC85E08093DE0183E0809311018091BF
:102C5000E10084FF37C08091E20084FF33C080E14F
:102C600089BD82E189BD09B400FEFDCF8091D80005
:102C70008F7D8093D8008091E1008F7E8093E1006A
:102C80008091E2008F7E8093E2008091E20081607B
:102C90008093E2008091DF01882311F084E007C077
:102CA0008091E30087FD02C081E001C083E0809352
:102CB000DE018091DE01843011F081E001C082E00C
:102CC000809311018091E10083FF2CC08091E2008C
:102CD00083FF28C08091E100877F8093E10082E03C
:102CE0008093DE011092DF018091E1008E7F80935E
:102CF000E1008091E2008E7F8093E2008091E2000B
:102D000080618093E20042E060E080E00E948611F2
:102D10008091F00088608093F00081E08093110141
:102D200080931001FF91EF91BF91AF919F918F918F
:102D30007F916F915F914F913F912F910F900FBEB7
:102D40000F901F9018952091E4003091E50095E6D2
:102D50004091EC00842F817040FF23C08091E800F7
:102D600080FD1DC08091DE01882399F0853099F0A7
:102D70008091EB0085FD11C04091E4005091E50089
:102D80002417350729F3915011F09A01E1CF84E01F
:102D9000089582E0089583E0089581E0089580E039
:102DA00008954091E80042FFDDCF089580E0089546
:102DB0009091B60192FF10C041E0282F2471243079
:102DC00009F040E031E0282F2871283009F030E088
:102DD000431711F02CE0822793FF10C041E0282F09
:102DE0002471243109F040E031E0282F2871283186
:102DF00009F030E0431711F02CE082273091B70141
:102E000030FF10C051E0282F2171213009F050E02F
:102E100041E0282F2871283009F040E0541711F0C4
:102E200029E0822731FF10C041E0282F2171213194
:102E300009F040E031E0282F2871283109F030E016
:102E4000431711F029E0822794FD877E0895823888
:102E5000910569F1B0F48133910509F475C048F426
:102E60008932910509F467C08A32910509F471C06D
:102E700008958533910509F459C089339105B9F056
:102E80000895833E910589F138F4803E9105D1F093
:102E9000823E910529F10895863E9105C9F1873E4C
:102EA0009105D9F1843E910509F06CC027C02091AD
:102EB000B60120FD57C021FD55C02091B70123FD6B
:102EC0005BC008958091B60180FD48C08091B70134
:102ED00080FF48C08091B60184FD46C083EE51C09A
:102EE0008091B60182FF3CC0F5CF8091B60182FD92
:102EF00037C08091B70180FD35C0ECCF8091B7011C
:102F000081FF36C08091B60184FD2EC087EE39C0A6
:102F10008091B60183FF2AC0F5CF8091B60183FD71
:102F200025C08091B70181FD23C0ECCF8091B6010F
:102F300085FD22C01FC08091B60185FD1BC0809118
:102F4000B70183FF19C00AC08091B60186FD16C083
:102F500017C08091B60186FD13C010C089E311C06F
:102F600082EE0FC080EE0DC080E00BC086EE09C07F
:102F700084EE07C085E305C089E203C08AE201C090
:102F800081E390E00895209128029091EF0157E0AD
:102F90002917A9F030E0529FF001539FF00D112442
:102FA000E051FE4F7181761306C07081781303C023
:102FB0007581741306C02F5F3F4F2770E9CF80E003
:102FC000089581E00895F894E82FE295EF70F0E01D
:102FD00031A1282F2F7081E090E001C0880F2A9541
:102FE000EAF7982F9095932391A392A1892B82A31E
:102FF00078940895AAE0B0E0E0E0F8E10C94EA2BC0
:10300000AE014F5F5F4F7A018AE0FA0111928A9513
:10301000E9F701E211E06A0196E2692E91E0792E6A
:1030200088248394912CF80180818F3F09F447C054
:10303000F894E82FE295EF70F0E021A18F70A401E1
:1030400002C0440F551F8A95E2F7CA01922F982BB0
:1030500091A392A18095892382A3789400C0E6E28F
:10306000F1E021E030E0A12CB12C41914F3F89F0FB
:10307000A42FA295AF70B0E090968C9190E04F7025
:1030800002C0959587954A95E2F780FD02C0C90177
:1030900002C080E090E0A82AB92A220F331F51E035
:1030A000E433F50711F7F80180818F3F11F00E949A
:1030B000E317F0EAFA95F1F7F601B182A0820F5F0B
:1030C0001F4FF2E0CF0ED11C6016710609F0ABCF96
:1030D0004AE050E0B7018AEA91E00E94612C892B16
:1030E00091F08AE0F701AAEAB1E001900D928A9589
:1030F000E1F781E0809339020E94651D90933802C8
:10310000809337020CC080913902882341F080916E
:103110003702909138020E944A1D059710F480E012
:1031200018C04AE050E06AEA71E087EC91E00E9442
:10313000612C892B59F08AE0EAEAF1E0A7ECB1E0D2
:1031400001900D928A95E1F781E001C080E0109234
:1031500039022A96EEE00C94062C753048F46E3055
:1031600038F4843028F4462F672F0E94CD1F08952D
:1031700080E090E008951F93CF93DF930E9427177C
:10318000EC01C11580E5D807E8F5C11590E4D90731
:1031900008F0A8C0C03ED10530F5CD3CD10508F0FF
:1031A00094C0C83AD10578F4C53AD10508F083C077
:1031B000C130D10509F47CC008F4F2C0C430D10597
:1031C00008F0F1C0EDC0C33CD10508F0E9C0C85A11
:1031D000D0E0CC0FDD1FCA5BDE4F0990D881C02D37
:1031E000CE019464E1C0C11580E2D80708F0CBC0DD
:1031F000C11591E0D90708F06BC0C83ED10508F4AD
:10320000D2C0CEC0C03682E5D80728F5C03492E5DA
:10321000D90708F079C0C03282E5D80708F06CC041
:10322000C11592E5D90708F481C04C2F4695469503
:1032300080E2489FA0011124C37021E030E0C90161
:1032400002C0880F991FCA95E2F7EA01C82BD92B53
:10325000CE019D68A9C0C03A82E5D807B8F48C2F8A
:103260008F71C03892E5D90708F07BC086958695A6
:1032700090E2899F90011124C37081E090E002C028
:10328000880F991FCA95E2F79A6868C0C03C82E52A
:10329000D80708F46DC0C03E92E5D90708F080C099
:1032A000CF71DD27DC2FCC27CE01806F906A7CC0E8
:1032B00081E090E079C0C55AD0E0CD5BDE4F8881D7
:1032C000C82FD0E0CE0190646FC0CE0190656CC075
:1032D0008D2F0E94D816182FCE0199270E942717EC
:1032E0001F715CC0CE0199270E942717CC27DF7081
:1032F000D06A8C2B9D2B58C0CF71D0E0DC2FCC270F
:10330000CE01816F906A50C08C2F8F718695869503
:1033100090E2899F90011124C37081E090E002C087
:10332000880F991FCA95E2F79C6818C08C2F8F717F
:103330000E94D81695E0D695C7959A95E1F7CF707B
:10334000D0E0DC2FCC27282F30E084FF05C084E0BC
:10335000220F331F8A95E1F7D069CE01822B932B80
:1033600023C090E0D82FCC27CE01846F906A1CC078
:103370008C2F8F710E94D8168F7190E0D82FCC2798
:10338000CE01906211C08D2F8F710E94D816182F18
:10339000CE0199270E9427171F719062912B04C0BC
:1033A00080E090E001C0CE01DF91CF911F910895A0
:1033B000A6E0B0E0EEEDF9E10C94F42B0E94651D5F
:1033C0008C0180913502909136020817190781F01F
:1033D00019821A820E94651D682F49815A81792FAE
:1033E00080E090E00E94BB291093360200933502E2
:1033F0002696E4E00C94102C809590913402892359
:103400008093340208959091340280912B02892B8D
:1034100090912A02992379F0892BECE3F2E027E0DE
:1034200090E0215029F031913323D9F39F5FF9CFF8
:10343000911110922A0280933A0248E050E06CE227
:1034400072E08AE392E00E94612C892BA9F088E067
:10345000EAE3F2E0ACE2B2E001900D928A95E1F786
:10346000E0916A02F0916B02309731F00280F381B3
:10347000E02D8AE392E009950895909129028095C4
:10348000892380932902282F277069F4981759F00F
:103490009091B70192FF07C08695869586950E9408
:1034A00047211092290208959091B70192FB22279B
:1034B00020F9281779F080FB92F99093B701609179
:1034C000B6017091B70184E090E00E94FF2A82E08B
:1034D0000E943D1A0895809128029091EF0189176A
:1034E00019F08F5F8770FBCF0895CF93DF938091A2
:1034F000EE0182958F7009F04EC08091ED01882316
:1035000009F449C0809128024091EF015091E901EE
:103510006091E801C091EA01D091EB0177E0841756
:10352000D1F190E0789FF001799FF00D1124DF0137
:10353000A051BE4F14962C911497222349F1119655
:103540002C911197251324C02C91261321C0159678
:103550002C91159721111CC012962D913C91139717
:103560002C1B3D0B283C310598F48091EE018F70A7
:1035700080618093EE01EA50FE4F80818F70806100
:10358000808388EE91E00E94110B0E946B1A03C0A9
:1035900001968770C4CFDF91CF910895A4E1B0E088
:1035A000E4EDFAE10C94EC2B8C0186E0F801DE01ED
:1035B0001F9601900D928A95E1F7F8018481E580CC
:1035C00098EE892E91E0992E9091EC01911120C0F6
:1035D000882309F463C1EE2009F442C0C8010E94A7
:1035E0006321F82E8823E1F187E0F801D4010190EE
:1035F0000D928A95E1F78091EC01813031F4809150
:10360000E8019091E9010E94CE200E94751A48C1FC
:10361000F801D080C180A280B380F090ED012091AC
:10362000EA013091EB01FF2009F4E7C0A501421B3C
:10363000530B483C510508F09DC0882309F430C164
:103640008091EE01282F207F9091E901222361F0E3
:103650009C1509F460C0C8010E946321811163C0F8
:10366000C8010E94110B1AC19C1113C09091E8016E
:103670009D110FC0E1100DC08F7080618093EE012D
:1036800088EE91E00E94110B8091EE01F801868393
:1036900003C1E1103AC040E06C2D8D2D0E94C3178C
:1036A00040E06C2D8D2D0E94C317E82E8111F4C0CF
:1036B000DF86C88A8F8598890E94CE20292F22957F
:1036C0002F70243020F49F70223028F009C02A5037
:1036D000223080F014C0992349F0811107C013C033
:1036E000992321F0F8019681907F69F0805E8830FF
:1036F00030F409C0803F38F0815F833020F0C8018A
:103700000E94110BEF2CFE2CCBC08091EE0181604A
:103710008093EE01C1C09091E8019D119CCFE11012
:103720009ACFF80198C0EE2009F49ACF2091EE01CB
:10373000822F82958F7090E002978CF08091E80143
:103740009091E90199878887BB86AA868091EC01D0
:103750008C871D862E87CE0108960E94110B87E06C
:10376000F801A8EEB1E001900D928A95E1F70E9470
:10377000751A94C09091EE01292F207F51F488EEA4
:1037800091E00E94110B87E0F40111928A95E9F70C
:1037900083C0882309F484C08091E9018C110CC096
:1037A0008091E8018D1108C0E11006C0F8019683F0
:1037B000C8010E94110B6AC0C8010E9463218823BE
:1037C00009F44ECFEE2009F44BCF2091EE01822F69
:1037D00082958F7090E0029714F28091E8019091A9
:1037E000E9019A838983BC82AB828091EC018D834D
:1037F0001E822F83CE010196B0CFA21AB30AF8EC35
:10380000AF16B10408F042C0882309F447C0FE2C6B
:10381000EE2009F425CF8091E9018C1129C0809117
:10382000E8018D1125C09091EE0190FD18C0892FFF
:1038300082958F70282F30E02115310581F0F80135
:1038400096832F30310541F08F5F982F9295907FAE
:1038500086818F70892B8683C8010E94110B87E0B7
:10386000F801A8EEB1E001900D928A95E1F718C039
:10387000C8010E946321811172CF8091EE018160A5
:103880008093EE01C8010E94110B0AC087E0F40189
:1038900011928A95E9F704C0F12C02C0FF24F39439
:1038A0008F2D6496ECE00C94082C9091B50121E0EA
:1038B00030E0F90101C0EE0F8A95EAF7D90102C0A4
:1038C000AA0FBB1F6A95E2F7BD016E2B01C0220F44
:1038D0004A95EAF7892F8623681303C0892F822B24
:1038E00003C02095822F89230E94442108950895C2
:1038F00080910F010895FC01EE0FFF1F8E0F9F1F97
:10390000FC01EA5BFD4F6183408322830895509A56
:1039100008958BB18E7F9BB191602FB7F894E6E448
:10392000F2E032E0E835F30789F0319148E09BB9E5
:10393000000000C037FF8BB9330F000000C000C08B
:1039400000C08BB900C04A9591F7EBCF2FBF8FE530
:1039500094E00197F1F700C0000008950F931F93C2
:10396000CF93DF938B01EA019091DE01943079F5DA
:103970008F708093E9008FEF9091E800815095FD62
:1039800006C095ED9A95F1F700008111F5CF809171
:10399000E80085FF1CC00E94A316882361F0809177
:1039A000E8008E778093E80012C0F80181918F01C2
:1039B0008093F1002197209791F38091E80085FD95
:1039C000F4CF8091E8008E778093E800E4CFDF9118
:1039D000CF911F910F910895CF93DF93EC0148E0B1
:1039E00050E0BC0181E00E94AE1C88E0FE01A4ED25
:1039F000B1E001900D928A95E1F7DF91CF910895A2
:103A000081E08093E00080E28093D8001092C900AA
:103A10008FE19EE40197F1F700C0000087E090EB92
:103A2000DC018093BE029093BF02A093C002B093CA
:103A3000C1029CE088E10FB6F894A89580936000DD
:103A40000FBE90936000FFCF78941F920F920FB635
:103A50000F9211248F939F93AF93BF9380916F0226
:103A600090917002A0917102B09172020196A11D15
:103A7000B11D80936F0290937002A0937102B09376
:103A80007202BF91AF919F918F910F900FBE0F90D7
:103A90001F9018959C014FB7F89480916F029091F8
:103AA0007002A0917102B09172024FBF821B930B02
:103AB00008952FB7F89460916F0270917002809111
:103AC0007102909172022FBF08952FB7F8948091E0
:103AD0006F0290917002A0917102B09172022FBF9B
:103AE00008951F920F920FB60F9211248F939F93F8
:103AF000AF93BF9380916E02811113C080916F02CA
:103B000090917002A0917102B09172024196A11D34
:103B1000B11D80936F0290937002A0937102B093D5
:103B20007202BF91AF919F918F910F900FBE0F9036
:103B30001F901895EAE3F2E09281891301C0128286
:103B4000319692E0E034F907B9F70895ACE3B2E0BA
:103B5000EFEF90E02D91821789F0EF3F19F42111DA
:103B600001C0E92F9F5F9630A9F7EF3F39F00E2E85
:103B7000000CFF0BE65CFD4F828308950895A3E0DF
:103B8000B0E0E5ECFDE10C94F62B20916C02309155
:103B90006D0228173907A1F090936D0280936C0293
:103BA000E0916A02F0916B02309751F024E0298392
:103BB0009B838A830084F185E02DCE0101960995CF
:103BC0002396E2E00C94122CA3E0B0E0EAEEFDE1D3
:103BD0000C94F62B2091680230916902281739075E
:103BE000A1F09093690280936802E0916A02F091DB
:103BF0006B02309751F023E029839B838A830084F2
:103C0000F185E02DCE01019609952396E2E00C9412
:103C1000122CE0916A02F0916B02309729F001902A
:103C2000F081E02D0995089580E0089587E290E005
:103C30000E94E12A0895CF93C82F811102C06FEF2F
:103C400001C065E284E290E00E94E12AC11102C055
:103C50006FEF01C061E085E290E00E94E12AC111AE
:103C600002C06FEF01C064E186E290E00E94E12AA9
:103C7000CF91089584E290E00E94BD2A853281F4BC
:103C800085E290E00E94BD2A813051F486E290E006
:103C90000E94BD2A91E0843109F090E0892F01C093
:103CA00080E0817008950F931F93CF93DF93C42F0B
:103CB000D22FFC0185818823B1F0409367020E94D6
:103CC000651D909366028093650280E28C0F8830B8
:103CD00008F068C0C77081E001C0880FCA95EAF794
:103CE0000E94B4215FC08091670248133DC080915B
:103CF0006502909166020E944A1D883C9105A0F5DC
:103D000010E21D0FCD17E9F080E28C0F883040F4EF
:103D1000C77081E001C0880FCA95EAF70E94AD2103
:103D2000183078F581E09D2F977001C0880F9A9523
:103D3000EAF70E94B421093351F560E570E089E3A8
:103D400029C0093319F460E570E002C060E070E05A
:103D5000802F0E948923183028F5D77081E001C098
:103D6000880FDA95EAF70AC080E28C0F8830D0F429
:103D7000C77081E001C0880FCA95EAF70E94AD21A3
:103D800011C0093351F460E570E089E309C060E0D7
:103D900070E0802F0E948923E0CF60E070E0802FE8
:103DA0000E948923DF91CF911F910F9108950E9466
:103DB000651D20916102211104C02091620222231D
:103DC00021F090935E0280935D02209163022111A5
:103DD00004C020916402222321F090935C0280931E
:103DE0005B02E0916A02F0916B02309749F082E049
:103DF00080935F020680F781E02D8FE592E00995C0
:103E0000089580915A0280FD16C081FD16C082FD82
:103E100018C080915902882391F0883290F428E0EC
:103E2000829FC001112468E270E00E94B62B862FA9
:103E3000672B29F007C082E0089584E0089581E0AF
:103E4000089588E0089580915A0280FD14C081FD94
:103E500014C082FD16C080915802882381F08E31F3
:103E600080F420E5829FC00111246EE170E00E9481
:103E7000B62B862F089584E1089588E2089588E09E
